:100000000C9438000C9455000C9455000C94550039
:100010000C9455000C9455000C9455000C9455000C
:100020000C9455000C9455000C9441020C9455000E
:100030000C9455000C944B070C9455000C945500EF
:100040000C94AA000C9455000C9455000C94680173
:100050000C9486020C9455000C9455000C94550099
:100060000C9455000C9455000C9455000C945500BC
:1000700011241FBECFEFD4E0DEBFCDBF11E0A0E062
:10008000B1E0E8E2F0E102C005900D92A039B107BD
:10009000D9F711E0A0E9B1E001C01D92A53FB10779
:1000A000E1F70E9438010C9412080C940000809132
:1000B0009201882331F480919401882311F4809176
:1000C0009601809398010E94FC05909191019923DB
:1000D00031F490919301992311F4909195018091BD
:1000E0009901882359F494304CF49D3F3CF0892FBA
:1000F0008E5F853030F480919001980F9093970136
:1001000014C0933031F480919001833061F486E023
:1001100007C09D3F41F4809190018D3F21F48AEF0B
:100120008093970102C01092970180919701819569
:100130000E94F10508951BBA8FEF8ABB85BB84BB73
:10014000C498BC9A84E181BF8AE083BF89B781608B
:1001500089BF08951F920F920FB60F9211242F930B
:100160003F934F935F936F937F938F939F93AF933F
:10017000BF93EF93FF9380910D018F5F80930D01EB
:10018000843079F510920D01A091ED01EA2FE295EE
:10019000EF70F0E0E050FF4F808180939D01B0E070
:1001A000AF70B070A050BF4F8C9180939C01A09114
:1001B000F101EA2FE295EF70F0E0E050FF4F80810F
:1001C00080939B01B0E0AF70B070A050BF4F8C9196
:1001D00080939A018091EE01882311F0C49801C0A8
:1001E000C49A50919A01E52FE37040919B01742FBE
:1001F00073702E2F220F220F272B30919C01632F1B
:100200006370220F220F262B90919D01220F220F47
:10021000892F8370282B9695969590939D01880F32
:10022000880F862B3695369530939C01880F880F62
:10023000872B4695469540939B01880F880F8E2B00
:100240005695569550939A0125BB80958BBBFF918F
:10025000EF91BF91AF919F918F917F916F915F913E
:100260004F913F912F910F900FBE0F901F901895B7
:100270008FEF8ABB84BB1BBA15BA0E945E010E9435
:10028000F9040E949B000E947D020E9433020E949A
:10029000A204809118010E949C0580E00E94C00584
:1002A0008091B3010E94C00578948091B9018823A0
:1002B000E1F31092B9010E944704F7CF82E080BDBC
:1002C00085E189B91AB886E880BD84E98AB90895BC
:1002D0001F920F920FB60F9211240F931F932F931B
:1002E0003F934F938F939F93EF93FF931AB11270A5
:1002F0000CB1E0911301F09114010994112309F05C
:10030000A4C00E3709F0A1C087E891E007C011230F
:10031000F9F401700093A00183E991E09093140136
:100320008093130192C0112399F40F7000939F01E1
:100330008BE991E0F3CF112359F080EA91E0EECF01
:10034000112331F0017000939E018BEA91E0E6CF1A
:100350008EE791E0E3CF8EE791E0909314018093D4
:100360001301112309F471C0202F2F703091A001C7
:1003700080911201831789F49091110180919F015E
:10038000981759F49091100180919E01981729F4C3
:1003900080910F01821709F458C0309312018091A7
:1003A0009F018093110140919E0140931001209381
:1003B0000F01882369F490910E01892F8195809314
:1003C0009101809190018330E9F4909391011AC0DA
:1003D000813051F410929101332311F48DEF01C05B
:1003E00083E0809390010EC0823019F480910E0159
:1003F00007C0843011F488E003C0883019F489E024
:1004000080939101332329F4809191018195809308
:100410009101222319F4109292010EC0223019F496
:1004200080910E0107C0243011F488E003C0283009
:1004300019F489E080939201442329F0809192017C
:100440008195809392010E945700FF91EF919F91B7
:100450008F914F913F912F911F910F910F900FBE50
:100460000F901F90189581B38F7081BB82B3806FFE
:1004700082BB87E282BD8DE087BD89B7806189BF7D
:1004800008951F920F920FB60F9211242F938F93FE
:100490009F9390B3907F80911601981719F09093D5
:1004A000160123C0809115018917F9F0292F94FDB9
:1004B00002C081E003C095FD04C08FEF80939601D8
:1004C00002C01092960126FD02C081E003C097FD94
:1004D00004C08FEF8093950102C0109295010E9495
:1004E000570080911601809315019F918F912F9154
:1004F0000F900FBE0F901F9018951CBE83E380B91C
:1005000011B886E88CBF88E981B908951F920F92CF
:100510000FB60F9211242F933F934F938F939F9376
:10052000EF93FF9343B18091A101882309F0EEC0BE
:10053000443409F478C0453410F54A3368F4403344
:1005400008F044C0433209F459C04D3209F45DC08B
:10055000463009F064C1D2C04E3309F45DC04F3358
:1005600038F44A3309F4CCC04C3309F058C151C0B7
:10057000423409F46AC0433409F051C10FC1443513
:1005800009F4A5C0453580F44C3409F452C04D340B
:1005900020F4473409F043C190C04D3409F477C0CA
:1005A000423509F03CC142C0473609F49DC0483687
:1005B00030F44535A9F1423609F031C13DC04D3620
:1005C00009F44FC0443709F02AC193C08091B001AB
:1005D0009091B1019C01220F331F220F331F220F74
:1005E000331F880F991F280F391F240F311D2053E7
:1005F00030403093B1012093B00136C11092B10167
:100600001092B0011092AF012FC181E08093AF0131
:100610002BC11092B20128C181E08093B20124C1A4
:100620008091B201AAC08091B201ABC08091B201A9
:10063000ACC08091B201ADC08091B0019091B10188
:100640009093CF018093CE0108C08091B00190912A
:10065000B1019093E0018093DF0181E08093B901C3
:1006600003C11092D0011092D1018091B0019091FC
:10067000B101892B91F38091AF01882321F081E0B2
:100680008093D101EACF81E08093D001E6CF109230
:10069000E1011092E2018091B0019091B101892BAA
:1006A000E1F28091AF01882321F081E08093E201A3
:1006B000D4CF81E08093E101D0CF8091B201882333
:1006C00011F483E001C081E080930E01C6CF8091D8
:1006D000AF01882321F08091B001819502C0809103
:1006E000B0010E94C005B9CF8091B001809318017C
:1006F000B4CF8091B2018093B401B6C080E590C0C0
:1007000081E08093A1011092A201AEC08091A2016C
:10071000433281F0E82FF0E0ED55FE4F40838F5FCC
:100720008093A201883009F09FC08FE383B91092B3
:10073000A1019AC01092A101882309F495C090915B
:10074000A301913549F1923509F44BC09D3409F06C
:1007500066C0823009F088C08091A4018E3661F0B5
:100760008F3624F4853609F057C00EC0833741F028
:10077000873709F051C00CC081E08093AE0182C080
:1007800081E08093AD017EC081E08093AB017AC0AF
:1007900081E08093AC0176C0813039F41092AB01D6
:1007A0001092AC011092AD0110C08230C1F5809161
:1007B000A4018E3651F08F361CF4853669F50BC0D6
:1007C000833731F0873741F509C01092AE015AC026
:1007D0001092AD0157C01092AB0154C01092AC0101
:1007E00051C0823009F040C08091A401873451F09B
:1007F00088341CF4833481F407C08D3439F0833598
:1008000059F408C081E003C083E001C088E0809310
:10081000170138C089E0FBCF8FE383B933C08FE382
:1008200083B922C08091170107C08091AD01882350
:1008300031F08091170181958093940102C010924C
:1008400094018091AB01882319F08091170107C0B2
:100850008091AC01882331F08091170181958093BC
:10086000930102C0109293010E945700FF91EF91F3
:100870009F918F914F913F912F910F900FBE0F90AD
:100880001F9018958091AE01882361F6CECFDF933B
:10089000CF93CDB7DEB72C970FB6F894DEBF0FBE5F
:1008A000CDBFF8948091D00189838091D1018A8352
:1008B0008091CE019091CF019C838B838091E10147
:1008C0008D838091E2018E838091DF019091E00120
:1008D00098878F8380910E0189878091B3018A87E1
:1008E000809118018B87789490E0FE0131969E01EB
:1008F000245F3F4F8191980FE217F307D9F79C8748
:10090000FE0131964E2F54E096E09E01245F3F4F4A
:100910008E2F841BE199FECF1FBA8EBB80818DBBC9
:10092000F8945CBB9CBB7894E217F30711F0319606
:10093000EFCF2C960FB6F894DEBF0FBECDBFCF9190
:10094000DF910895DF93CF93CDB7DEB72C970FB625
:10095000F894DEBF0FBECDBFFE0131964E2F91E061
:100960009E01245F3F4F8E2F841BE199FECF1FBA5B
:100970008EBB9CBB8DB38083E217F30711F03196D9
:10098000F2CF90E0FE0131969E01245F3F4F8191AE
:10099000980FE217F307D9F78C85891709F5898134
:1009A0008093D0018A818093D1018B819C81909327
:1009B000CF018093CE018D818093E1018E81809360
:1009C000E2018F8198859093E0018093DF01898512
:1009D00080930E018A858093B3018B8580931801E3
:1009E0002C960FB6F894DEBF0FBECDBFCF91DF912E
:1009F00008951092ED011092EE018DEE91E090932A
:100A0000CD018093CC011092F10181EF91E09093A0
:100A1000DE018093DD0189B7806489BF08956F92FC
:100A20007F928F929F92AF92BF92CF92DF92EF927E
:100A3000FF920F931F93CF93DF93EC01E62ECA0131
:100A4000B9010E94B6075B016C01FF2400E010E0D1
:100A5000C801B7010E94B6077B018C019595879567
:100A6000779567956A0D7B1D8C1D9D1DA8019701CB
:100A70000E94D507922E832E742E652E622F732F1F
:100A8000842F952FA80197010E94B6079B01AC0106
:100A90002A193B094C095D09C601B5010E94D50719
:100AA00079018A01292D382D472D562DC901DA01EA
:100AB000883E23E0920720E0A20720E0B20724F45A
:100AC00088EE93E0A0E0B0E09983888317FD11C021
:100AD0001C8280E0E81680E0F80681E0080780E0EC
:100AE00018071CF020E030E001C097013B832A8307
:100AF00014C081E08C8321E0E21620E0F2062FEFA3
:100B000002072FEF12071CF480E090E004C0882752
:100B100099278E199F099B838A83DF91CF911F911B
:100B20000F91FF90EF90DF90CF90BF90AF909F908C
:100B30008F907F906F900895FF920F931F93F82EE0
:100B40000AEB11E024E930E541E050E0682FC801EC
:100B50000E940F0520E831E541E050E06F2DC8010B
:100B600005960E940F052DED3CE541E050E06F2D0C
:100B7000C8010A960E940F051F910F91FF900895DA
:100B80008093B30187FF04C081E0809399010895A9
:100B9000833030F510929901992787FD9095FC01DB
:100BA000EE0FFF1FEE0FFF1FE80FF91FE654FE4F79
:100BB000808191819BBD8ABD1DBC1CBC1FBC89E08E
:100BC0008EBD1092F0011092EF018281938190937B
:100BD000F4018093F30184818093C9011092CA01CA
:100BE0000895982F8091DA01882319F481E0809389
:100BF000DA019093CB010895982F8091EB0188231F
:100C000019F481E08093EB019093DC010895E62FC5
:100C1000F0E0EE0FFF1FE758FE4F2081FC01278711
:100C20000895CF93DF93EC0189859A85892B21F470
:100C300087E296E09A8789878D81882329F08E81C3
:100C4000882311F01E821D82E985FA850994888126
:100C5000882381F48E81882309F062C08091790114
:100C60008F87E981FA811082E981FA81118287E216
:100C700096E015C018160CF490C052C088818823E5
:100C800089F48D81882381F4809179018F87E981AE
:100C9000FA811082E981FA8111828EE396E09A87C7
:100CA0008987F6C087FDB2C08B819C81892B79F240
:100CB00020918E011C861B8680918D018F8721FDDE
:100CC00003C089E591E009C08091B401882319F43B
:100CD00089E191E002C089E391E09E878D87E981F7
:100CE000FA812170218387E796E09A878987A98115
:100CF000BA818F81ED85FE85E80FF11D80818C938F
:100D00008F818F5F8F718F838B859C8501969C87E8
:100D10008B872B813C812817390708F498CFB8C0FE
:100D20008B819C81892B09F4A9CF20918E011C868F
:100D30001B8680918D018F8721FD03C089E591E09D
:100D400009C08091B401882319F489E191E002C0BF
:100D500089E391E09E878D87E981FA812170218363
:100D600084EB96E09A878987A981BA818F81ED8586
:100D7000FE85E80FF11D80818C938F8181508F71EA
:100D80008F838B859C8501969C878B872B813C81EB
:100D90002817390708F472CF7BC0E82FFF27E7FD3B
:100DA000F095EE0FFF1FE758FE4F2181E82FF0E08E
:100DB000EE0FFF1FE758FE4F80818F8721FD03C094
:100DC00089E591E009C08091B401882319F489E193
:100DD00091E002C089E391E09E878D87E981FA81E5
:100DE0002170218385EF96E03CC098858881981713
:100DF00009F02DCFA981BA818F81ED85FE85E80F9D
:100E0000F11D80818C938F818F5F40C0E82FFF2779
:100E1000E7FDF095EE0FFF1FF095E195FF4FE758C6
:100E2000FE4F21818195E82FF0E0EE0FFF1FE7587C
:100E3000FE4F80818F8721FD03C089E591E009C0C5
:100E40008091B401882319F489E191E002C089E31B
:100E500091E09E878D87E981FA812170218386E365
:100E600097E09A8789878881888712C098858881CA
:100E7000981709F003CFA981BA818F81ED85FE858E
:100E8000E80FF11D80818C938F8181508F718F834A
:100E9000DF91CF9108951F920F920FB60F921124F8
:100EA0002F933F938F939F932091EF013091F00107
:100EB0002F5F3F4F3093F0012093EF018091C901E4
:100EC0009091CA01892B71F08091F3019091F40106
:100ED000009741F02817390728F01092F00110927E
:100EE000EF013BC09091DA01992369F08091DB0119
:100EF0008F5F8093DB01891730F01092DB018BEC60
:100F000091E00E9411069091EB01992369F0809184
:100F1000EC018F5F8093EC01891730F01092EC01A7
:100F20008CED91E00E9411068091C9019091CA0157
:100F3000892B99F42091F3013091F40121153105A9
:100F400061F08091EF019091F0018217930728F0F2
:100F50001092F0011092EF01C5CF9F918F913F91B8
:100F60002F910F900FBE0F901F901895629FD00188
:100F7000739FF001829FE00DF11D649FE00DF11D54
:100F8000929FF00D839FF00D749FF00D659FF00D03
:100F90009927729FB00DE11DF91F639FB00DE11DF0
:100FA000F91FBD01CF011124089597FB092E0526D5
:100FB0000ED057FD04D014D00AD0001C38F4509540
:100FC0004095309521953F4F4F4F5F4F0895F6F76D
:100FD00090958095709561957F4F8F4F9F4F0895A5
:100FE000A1E21A2EAA1BBB1BFD010DC0AA1FBB1F2D
:100FF000EE1FFF1FA217B307E407F50720F0A21B9F
:10100000B30BE40BF50B661F771F881F991F1A940B
:1010100069F760957095809590959B01AC01BD0135
:08102000CF010895F894FFCF01
:1010280000011115550000000002222AAA0303FF3F
:10103800FFFFFF7E01F0F00184041424344443428E
:101048004140494A4B4C3C2C1C0C9CACBCCCCBCAF8
:10105800C9C0C1C2C3C4B4A4944444444440404039
:10106800404C4C4C4C0C0C0C0CCCCCCCCCC0C0C068
:10107800C0C4C4C4C40404040444444444444444AC
:10108800444C4C4C4C4C4C4C4CCCCCCCCCCCCCCC20
:10109800CCC4C4C4C4C4C4C4C4010290024802304D
:1010A8000224021C0218030C0306030301030000B8
:00000001FF
